:10000000DDC2D5C0D8C035C218951895EBC118957A
:0A001000ABC01895189518951895C7
:10002000D7C05EC1EAC06FC145C14CC147C14EC116
:1000300071C174C177C19EC19FC1A3C1A4C1ABC12D
:10004000ADC166C165C164C163C1ABC19EC1A0C180
:1000500041C1F9C0FAC0FCC0FDC0FEC000C102C170
:100060000CC138C137C136C135C134C133C132C109
:1000700013B290B3E894B699689495F9907E089578
:1000800015BA089508950895979806C029D09798AD
:1000900003C026D0979A00C08F9A8E9A969845BB37
:1000A0004FEF44BBC39A0000000000000000C3985B
:1000B00040E045BB44BB97988F988E9808959798D9
:1000C00002C0979A00C08F9A8E9A969AC39A00009F
:1000D00000000000000043B3C3988F988E980895E5
:1000E0008F9A8E9A9798969A4F9340E9419542BF7E
:1000F00042E048BF48B741FD08C0C398C39A00001A
:100100000000000000009F99F5CFC398969897983B
:100110008F988E984F91089569B36095089566B34E
:10012000629564FB61F965FB60F96370089546E1CF
:1001300042BB41E341BB929840E045BB40E044BB39
:1001400043E848BB4CEB47BB4FEF4BBB40E04ABBDF
:1001500042EA4FBDF8942F93207419F0C29A2F9160
:100160000895C2982F91089501D01895829B04C0DC
:10017000BD1308C0AC1306C03FB66E986C982B7FB9
:100180003FBE08956C9A6E9A3D903FB83FB624608A
:10019000B1FDA0E6B17027FD07C020685A95503820
:1001A00020F42064D7DF01C02F773FBE089522FDE1
:1001B0001895DCDF18954FB65BDF51F0F0E0E0E01A
:1001C00096FBE0F997FBE1F995FBE2F9709609944B
:1001D000C4985F3C71F01992D1FDC0E6D17027FF41
:1001E00003C02F77539505C020685E3B10F02F7B2E
:1001F000B1DF22FD6FC0BADF6DC0C49817FC1BC011
:1002000016FC68C015FC18C014FC42C013FC42C0A8
:1002100012FCD4C111FE949811FE8C9A11FC8C989A
:1002200011FC949A10FE919810FE899A10FC8998FE
:1002300010FC919A4FC04EC0F0E0E12DEF70B896DF
:10024000109008020994C12C45C010920C0242C0C3
:100250001EBA40C01FBA3EC01DBA46D23BC01DBA2E
:1002600048D238C010920A02E0E0889417FC089443
:10027000111CEE1FEBBD1ABC2DC010920B02E0E06A
:10028000889417FC0894111CEE1FE9BD18BC22C00D
:10029000712C20C0E0E010FCEFEFF0E010FCF1E08A
:1002A000E0930B02F9BDE8BD11FA34F912FA35F901
:1002B00051DF10C0C498412DE9DE0CC0C498412D17
:1002C000E8DE08C0C4981092080204C0C4981092D6
:1002D000090200C07894839BFECF4FBEC49A189544
:1002E0006894819BE89410F826FB11F820FB12F823
:1002F00021FB13F824FB14F823FB15F825FB16F853
:10030000E89417F851C0F0E0E72DEF707896099463
:1003100011244AC01A2C2F7E1DDF46C01B2C2F7EB5
:1003200019DF42C010900002E32FEF7001F13A95FF
:10033000E130E9F0E0910102E0930002E091020275
:10034000E0930102E0910302E0930202E0910402D3
:10035000E0930302E0910502E0930402E0910602BB
:10036000E0930502E0910702E09306021DC0277F9B
:10037000F1DE1AC0152E18C01E2C2F7DEE24EADEE9
:1003800013C0BCD111C0BDD10FC099DE142E0CC05A
:1003900098DE142E09C010900A0206C010900B02BD
:1003A00003C01090100000C04F924424409444BAFF
:1003B00015BA66DE67DEC498789483990BC0869977
:1003C000FCCFC49A839906C0869BFCCF169458DE56
:1003D000C498F3CF58DE442444BA45BA4F904FBE78
:1003E000C49A18956FB698DE68112224862E97DE7F
:1003F00069112224962E27FE239464E06FBE6211B9
:100400001895682D6D1559F0D62EE32FEF70E3FF88
:100410003395E3FDEA95F2E0608328609BDE7894F3
:10042000692D6227637011F46FBE1895692D660FF0
:10043000660F622B6F702C7F29296230A9F064301F
:1004400099F06D3089F06B3079F0613041F06730B0
:1004500031F06E3021F0683011F06FBE1895EA94DB
:10046000206278DE6FBE1895E394206273DE6FBE63
:1004700018950FB68EB570E478277EBD72B780E010
:1004800082BF789488B781FF06C00027FF24112718
:1004900082E088BF79E10FBE17FD1895743180F0B6
:1004A000713224F410D060F00FBE1895793240F00C
:1004B0007E3334F408D020F006D010F00FBE18952B
:1004C0001FEF0FBE18958EB5809586FB139510FD16
:1004D00012C086F981278074B9F01234A9F014345F
:1004E00099F087F9881FFF1C001F1C3191F01C3503
:1004F00059F08894089516F91B3541F01D3121F00B
:100500001D3511F088940895089408958894FF1C6F
:10051000001FAF2CFF1C001FFF1C001F05FBA6F8CF
:100520000F71B02E6894BC10E894A7F8206112DE19
:1005300008940895AF93A2E0AA95F1F7AF910895BA
:10054000AF93A1E0AA95F1F7AF910895BC2F9198D0
:10055000899AF6DF0894BB1F01C0BB0F79F094980D
:100560008C9A20F400008998919A03C09198899AF6
:1005700000C0E0DF8C98949ADDDFEFCF94988C9ADE
:100580008998919AD7DF8C98949A849BFECF88940F
:1005900081990894CFDF0895DDCF94988C9A919833
:1005A000899AC8DF8C98949ACBDF8998919AC2DF98
:1005B00008958C988998949A919A08954FE54DBF23
:1005C00042E04EBFB4DDA0E6BB27C0E6DD275527DD
:1005D00049E84DB94EB14BE045BF40EC4BBF44E05C
:1005E00043BF1FEF41E04EBD48E849BFBB24AA24EA
:1005F000CC24DD24EE2477243327F89A4DEF4EBB2C
:1006000083D0E0E0EBBD4ABD7FD0E0E0889447FDB9
:100610000894441FEE1FE9BD48BD76D0403051F12B
:100620004FEF58D046E756D043E054D048E32EDD94
:1006300048E32CDD46E02ADD4CE028DD41E026DD04
:100640004DB34F3FB9F040E04FBB4EBB40E41EDD21
:1006500040E443D040E81ADD40E13FD040EC16DDF5
:1006600040E13BD040E912DD40E137D040ED0EDD06
:1006700040E133D040E0842E52DD962E292D2064B7
:10068000909ACF93BF93C79894DFCAE35FDFB8E631
:1006900083DFB3E981DFB0EB7FDFB0E07DDFB2E085
:1006A0007BDF7BDFCAE352DFB8E676DFB0E074DFE2
:1006B000B1E072DF72DFC79ABF91CF917894C49A8C
:1006C000C29AFFCF419542BF42E048BF48B741FFC1
:1006D000FDCF0895F7DF48E3D7CC4F9315D0D9DC91
:1006E0004F914A95D1F70895E29AE19AE199FECFA8
:1006F0000895E29AE19AE199FECF09C0E09A1DB20D
:100700000895E09A1DB203C0E09A4DB300C0EEB365
:10071000FFB33196EEBBFFBB0895EEB3FFB3319745
:06072000EEBBFFBB0895D3
:00000001FF
